:020000040000FA
:06000000703002303A28C6
:08000800A000030EA100831209
:1000100081018B100B11210E8300A00E200E090010
:0C007400203084008001840A6030040207
:10008000031C3C281230B0002B218316FF23900064
:10009000831283160C308505870183128501870141
:1000A000073099000030831691009F008312C830FA
:1000B00083168100831231309000003083168C004B
:1000C000831210308B00792181018E018F010B1179
:1000D0008B100B108C018B178020311982200F217F
:1000E000B30B7E28031085190314B90DF0303902C3
:1000F000031982210F30390203197E2186216C28D1
:1001000064000800080031110130B7008B13203063
:10011000370783169B001C141A088312A4001030A2
:10012000370783169B001C141A088312A3000030A3
:10013000370783169B001C141A088312A2008B1722
:10014000321CA82822090339A200A309A409A50981
:1001500001303702031DB1283D18B1283D143E146B
:10016000522101303702031DBA283D1CBA283D1028
:100170003E147621BB28B70A023037020318080064
:1001800086280130B600B300B400B500B700850181
:100190008701B1138020B30BE728031085190314DE
:1001A000B90DF030390203190529B41F8501B41FB8
:1001B0008701B40BE7283708B6080319B6000319FE
:1001C000E528FF3085008700B6039630B400311D66
:1001D000CA283111321CF1282D090339AD00AE09AE
:1001E000AF098B1320303707BB002F08BA00182146
:1001F00010303707BB002E08BA001821003037072F
:10020000BB002D08BA0018218B1785018701B70A9A
:10021000B60102303702031CCA28792108003E1CAF
:1002200008003E101030BB003D08BA00182108003D
:100230008B133A0883161C159A003B089B00553017
:100240009D00AA309D009C1464009C1824291C1158
:1002500083128B170800831610309B001C141A0899
:100260008312BD00831620309B001C141A088312D1
:10027000DF00831670309B001C141A088312D6000E
:100280000E07D7005707D8005607DB005807DA00DB
:100290005607D9005807D5007030BB005708BA0080
:1002A000182108000130BD000430C200C50005302F
:1002B000C400C600CA000730C100C300C700C800A0
:1002C000C9005F19C1175F19C2175F19C317DF197A
:1002D000C4175F1AC5175F1AC6175F1AC7175F1AC8
:1002E000C8175F1BC917DF18CA17080085018701E7
:1002F0000800851DB9033D18522108003D143E1425
:10030000522108003D103E147621080001303D05C1
:10031000031908005F198E295C1805165F199229C8
:10032000DC1885165F1996295C190514DF199A29BE
:10033000DC1985145F1A9E295C1A87145F1AA2299A
:10034000DC1A07155F1AA6295C1B07145F1AAA2975
:10035000DC1B87165F1BAE295D180716DF18B22954
:10036000DD188715E6300E02031CCA295F1D05162D
:100370005F1D85165F1D0514DF1D85145F1E871424
:100380005F1E07155F1E07145F1E87165F1F071687
:10039000DF1C87158F08031908008F01850187016D
:1003A0005508DE00C823D5005608DE00C823D60055
:1003B0005708DE00551CC823D7005808DE00D51C9E
:1003C000C823D8005908DE00551DC823D9005A0893
:1003D000DE00D51DC823DA005B08DE00551EC823E9
:1003E000DB005F1D0D2AC11B082AC11C0512C11CA0
:1003F000FC29051258190516CB0B1E2A5608CB00EE
:10040000C101D51BC114D81BC1105818C1101E2A18
:100410000512CB0B1E2AC1031E2AC108031905169B
:1004200003191E2ACB0B1E2AD51BC1035508CB006E
:10043000D5185C14D51E5C10D51D5C105F1D3A2AC2
:10044000C21B352AC21C8512C21C292A85125818C3
:100450008516CC0B4B2A5608CC00C201D61BC21401
:100460005A18C210D619C2104B2A8512CC0B4B2A2F
:10047000C2034B2AC2080319851603194B2ACC0B59
:100480004B2AD61BC2035608CC00D61ADC14561DC4
:10049000DC10561FDC105F1D672AC31B622AC31CB9
:1004A0000510C31C562A05105A190514CD0B782ABD
:1004B0005708CD00C301D71BC314D51AC310D719D1
:1004C000C310782A0510CD0B782AC303782AC308F5
:1004D000031905140319782ACD0B782AD71BC303F7
:1004E0005708CD00571A5C15571F5C11D71D5C11BA
:1004F000DF1D942AC41B8F2AC41C8510C41C832AA8
:100500008510D51B8514CE0BB02A5808CE00C40127
:10051000D81BC414D71AC410D819C410B02A851017
:10052000CE0BB02AC403B02ADF1F9F2ACE0BB02AFD
:100530005808CE00D51BDC15DA1FDC11B02AC40820
:10054000031985140319B02ACE0BB02AD81BC40393
:100550005808CE00581ADC15D81FDC11D81DDC1144
:100560005F1ECC2AC51BC72AC51C8710C51CBB2A09
:100570008710D51A8714CF0BDD2A5908CF00C50183
:10058000D91BC514561AC510D81BC510DD2A8710F3
:10059000CF0BDD2AC503DD2AC5080319871403190B
:1005A000DD2ACF0BDD2AD91BC5035908CF00D91B83
:1005B0005C16D91F5C12D91C5C125F1EF92AC61B7F
:1005C000F42AC61C0711C61CE82A0711D71A0715FA
:1005D000D00B0A2B5A08D000C601DA1BC614D51A54
:1005E000C610D619C6100A2B0711D00B0A2BC6034A
:1005F0000A2BC6080319071503190A2BD00B0A2B5F
:10060000DA1BC6035A08D0005A1ADC165A1EDC122E
:10061000DA1FDC125F1E262BC71B212BC71C0710FD
:10062000C71C152B071059190714D10B372B5B0862
:10063000D100C701DB1BC714D719C710DB19C710BE
:10064000372B0710D10B372BC703372BC7080319DC
:1006500007140319372BD10B372BDB1BC7035B08A0
:10066000D100DB195C17DB1D5C135B1E5C135F1E86
:10067000532BC81B4E2BC81C8712C81C422B871239
:1006800058198716D20B642B5608D200C801D91B03
:10069000C8145A19C810551AC810642B8712D20BE7
:1006A000642BC803642BC808031987160319642B2D
:1006B000D20B642BD71BC8035908D200561ADC177B
:1006C000561EDC13DA1FDC135F1F802BC91B7B2B2C
:1006D000C91C0712C91C6F2B071255190716D30B1B
:1006E0009A2B5808D300C901D61BC914D91AC910AE
:1006F000D819C9109A2B0712D30B9A2BC9039A2B1E
:100700005F1C8B2BD30B9A2B5708D300D61B5D1481
:10071000D81F5D109A2BC9080319071603199A2BC5
:10072000D30B9A2BD51AC9035808D300D61B5D14D6
:10073000D81F5D10DF1CB62BCA1BB12BCA1C87113A
:10074000CA1CA52B8711D51B8715D40B080055088B
:10075000D400CA01D51BCA14561ACA10D619CA1019
:1007600008008711D40B0800CA030800CA0803193F
:10077000871503190800D40B0800D81BCA035608B4
:10078000D400591ADD14591EDD10DA1FDD100800DF
:10079000C001DE080319DE035E184014DE1A40149F
:1007A0004008C0015E1C4014DE1E4014C005C00C91
:0407B0005E0C0800D3
:084000000D000300060005009D
:02400E00CC01E3
:10420000FF00FF00FF00FF00FF00FF00FF00FF00B6
:10421000FF00FF00FF00FF00FF00FF00FF00FF00A6
:104220000100FF00FF00FF00FF00FF00FF00FF0094
:10423000FF00FF00FF00FF00FF00FF00FF00FF0086
:104240000300FF00FF00FF00FF00FF00FF00FF0072
:10425000FF00FF00FF00FF00FF00FF00FF00050060
:10426000FF00FF00FF00FF00FF00FF00FF00FF0056
:10427000FF00FF00FF00FF00FF00FF00FF00FF0046
:10428000FF00FF00FF00FF00FF00FF00FF00FF0036
:10429000FF00FF00FF00FF00FF00FF00FF00FF0026
:1042A000FF00FF00FF00FF00FF00FF00FF00FF0016
:1042B000FF00FF00FF00FF00FF00FF00FF00FF0006
:1042C000FF00FF00FF00FF00FF00FF00FF00FF00F6
:1042D000FF00FF00FF00FF00FF00FF00FF00FF00E6
:1042E0000200BA00FF00FF00FF00FF00FF00FF0018
:1042F000FF00FF00FF00FF00FF00FF00FF000000C5
:00000001FF
